:020000020000FC
:020000007FC2BD
:02001C00C5C25B
:10010000808386898C8F9295989C9FA2A5A8ABAE80
:10011000B0B3B6B9BCBFC1C4C7C9CCCED1D3D5D892
:10012000DADCDEE0E2E4E6E8EAECEDEFF0F2F3F54B
:10013000F6F7F8F9FAFBFCFCFDFEFEFFFFFFFFFF00
:10014000FFFFFFFFFFFFFEFEFDFCFCFBFAF9F8F7E7
:10015000F6F5F3F2F0EFEDECEAE8E6E4E2E0DEDCFF
:10016000DAD8D5D3D1CECCC9C7C4C1BFBCB9B6B318
:10017000B0AEABA8A5A29F9C9895928F8C898683E0
:10018000807C797673706D6A6763605D5A575451ED
:100190004F4C494643403E3B383633312E2C2A27BC
:1001A0002523211F1D1B1917151312100F0D0C0AE3
:1001B000090807060504030302010100000000000E
:1001C0000000000000000101020303040506070807
:1001D000090A0C0D0F1012131517191B1D1F2123CF
:1001E00025272A2C2E313336383B3E404346494C96
:1001F0004F5154575A5D6063676A6D707376797CAE
:10020000000102030405060708090A0B0C0D0E0F76
:10021000101112131415161718191A1B1C1D1E1F66
:10022000202122232425262728292A2B2C2D2E2F56
:10023000303132333435363738393A3B3C3D3E3F46
:10024000404142434445464748494A4B4C4D4E4F36
:10025000505152535455565758595A5B5C5D5E5F26
:10026000606162636465666768696A6B6C6D6E6F16
:10027000707172737475767778797A7B7C7D7E7F06
:10028000808182838485868788898A8B8C8D8E8FF6
:10029000909192939495969798999A9B9C9D9E9FE6
:1002A000A0A1A2A3A4A5A6A7A8A9AAABACADAEAFD6
:1002B000B0B1B2B3B4B5B6B7B8B9BABBBCBDBEBFC6
:1002C000C0C1C2C3C4C5C6C7C8C9CACBCCCDCECFB6
:1002D000D0D1D2D3D4D5D6D7D8D9DADBDCDDDEDFA6
:1002E000E0E1E2E3E4E5E6E7E8E9EAEBECEDEEEF96
:1002F000F0F1F2F3F4F5F6F7F8F9FAFBFCFDFEFF86
:1003000000020406080A0C0E10121416181A1C1EFD
:1003100020222426282A2C2E30323436383A3C3EED
:1003200040424446484A4C4E50525456585A5C5EDD
:1003300060626466686A6C6E70727476787A7C7ECD
:1003400080828486888A8C8E90929496989A9C9EBD
:10035000A0A2A4A6A8AAACAEB0B2B4B6B8BABCBEAD
:10036000C0C2C4C6C8CACCCED0D2D4D6D8DADCDE9D
:10037000E0E2E4E6E8EAECEEF0F2F4F6F8FAFCFE8D
:10038000FFFDFBF9F7F5F3F1EFEFEBE9E7E5E3E16B
:10039000DFDDDBD9D7D5D3D1CFCFCBC9C7C5C3C15B
:1003A000BFBDBBB9B7B5B3B1AFAFABA9A7A5A3A14B
:1003B0009F9D9B99979593918F8F8B89878583813B
:1003C0007F7D7B79777573716F6F6B69676563612B
:1003D0005F5D5B59575553514F4F4B49474543411B
:1003E0003F3D3B39373533312F2F2B29272523210B
:1003F0001F1D1B19171513110F0F0B0907050301FB
:1004000000000000000000000000000000000000EC
:1004100000000000000000000000000000000000DC
:1004200000000000000000000000000000000000CC
:1004300000000000000000000000000000000000BC
:1004400000000000000000000000000000000000AC
:10045000000000000000000000000000000000009C
:10046000000000000000000000000000000000008C
:10047000000000000000000000000000000000007C
:10048000FFFFFFFFFFFFFFFFFFFFFFFFFFFFFFFF7C
:10049000FFFFFFFFFFFFFFFFFFFFFFFFFFFFFFFF6C
:1004A000FFFFFFFFFFFFFFFFFFFFFFFFFFFFFFFF5C
:1004B000FFFFFFFFFFFFFFFFFFFFFFFFFFFFFFFF4C
:1004C000FFFFFFFFFFFFFFFFFFFFFFFFFFFFFFFF3C
:1004D000FFFFFFFFFFFFFFFFFFFFFFFFFFFFFFFF2C
:1004E000FFFFFFFFFFFFFFFFFFFFFFFFFFFFFFFF1C
:1004F000FFFFFFFFFFFFFFFFFFFFFFFFFFFFFFFF0C
:100500000FED0DBF03E209B908E90AB978940FEFBE
:1005100007BBF1E0E0E0D0E0C0E085E595E3A0E0D6
:10052000C80FD91FEA1FC89508BAFACF0BB107FF49
:10053000FDCF0CB108950F930BB105FFFDCF0F91C7
:100540000CB908950F9306E4F6DF0027F4DF0A2FB5
:10055000F2DF092FF0DF082FEEDF0AE0ECDF0F916A
:10056000089501967727A71F08950A967727A71F52
:10057000089574E6870F7727971FA71F089501979F
:100580007727A70B08950A977727A70B0895772752
:100590008456970BA70B0895C9DFC8DFA02FC6DFCD
:1005A000902FC4DF802F08950F930CB10B3211F4FC
:1005B000D8DF2FC0053711F4D8DF2BC0053511F473
:1005C000D8DF27C00D3211F4DADF23C0043611F46E
:1005D000DADF1FC0043411F4DADF1BC0033711F473
:1005E000DBDF17C00F3309F414C0013319F4F1E055
:1005F000E0E00FC0023319F4F2E0E0E00AC0033398
:1006000019F4F3E0E0E005C0043319F4F4E0E0E0AD
:0806100000C098DF0F9118955E
:00000001FF
